
 STORAGE

 Start     Length     Name                   Class
 0001:0000 0014CH     SEG_CODE_TEXT          CODE
 0001:0150 0007FH     _TEXT                  CODE
 0002:0000 00010H     NULL                   BEGDATA
 0002:0010 00006H     _DATA                  DATA
 0002:0016 00000H     CDATA                  DATA
 0002:0016 00000H     XIFB                   DATA
 0002:0016 00000H     XIF                    DATA
 0002:0016 00000H     XIFE                   DATA
 0002:0016 00000H     XIB                    DATA
 0002:0016 00000H     XI                     DATA
 0002:0016 00000H     XIE                    DATA
 0002:0016 00000H     XPB                    DATA
 0002:0016 00000H     XP                     DATA
 0002:0016 00000H     XPE                    DATA
 0002:0016 00000H     XCB                    DATA
 0002:0016 00000H     XC                     DATA
 0002:0016 00000H     XCE                    DATA
 0002:0016 00000H     XCFB                   DATA
 0002:0016 00000H     XCF                    DATA
 0002:0016 00000H     XCFE                   DATA
 0002:0016 0000CH     DBDATA                 DATA
 0002:0022 00000H     CONST                  CONST
 0002:0022 00019H     HDR                    MSG
 0002:003B 00082H     MSG                    MSG
 0002:00BD 00002H     PAD                    MSG
 0002:00BF 00001H     EPAD                   MSG
 0002:00C0 00000H     _BSS                   BSS
 0002:00C0 00000H     XOB                    BSS
 0002:00C0 00000H     XO                     BSS
 0002:00C0 00000H     XOE                    BSS

 Origin   Group
 0002:0   DGROUP

 Address   Export                  Alias

 0001:000C DLLGETCLASSOBJECT       DLLGETCLASSOBJECT
 0001:0032 STGCREATEDOCFILE        STGCREATEDOCFILE
 0001:0058 STGCREATEDOCFILEONILOCKBYTES  STGCREATEDOCFILEONILOCKBYTES
 0001:00DA STGISSTORAGEFILE        STGISSTORAGEFILE
 0001:0100 STGISSTORAGEILOCKBYTES  STGISSTORAGEILOCKBYTES
 0001:007E STGOPENSTORAGE          STGOPENSTORAGE
 0001:00AC STGOPENSTORAGEONILOCKBYTES  STGOPENSTORAGEONILOCKBYTES
 0001:0126 STGSETTIMES             STGSETTIMES
 0001:0006 WEP                     WEP

  Address         Publics by Name

 0000:0000  Imp  CALLOBJECTINWOWCHECKTHKMGR (COMPOBJ.204)
 0000:0000  Imp  CALLPROC32W          (KERNEL.CALLPROC32W)
 0001:000C       DLLGETCLASSOBJECT
 0000:0000  Imp  FREELIBRARY32W       (KERNEL.FREELIBRARY32W)
 0000:0000  Imp  GETPROCADDRESS32W    (KERNEL.GETPROCADDRESS32W)
 0000:0000  Imp  GETVDMPOINTER32W     (KERNEL.GETVDMPOINTER32W)
 0001:0000       LIBMAIN
 0000:0000  Imp  LOADLIBRARYEX32W     (KERNEL.LOADLIBRARYEX32W)
 0000:0000  Imp  OUTPUTDEBUGSTRING    (KERNEL.115)
 0000:0008  Abs  pAtomTable
 0000:0006  Abs  pLocalHeap
 0000:000E  Abs  pStackBot
 0000:000C  Abs  pStackMin
 0000:000A  Abs  pStackTop
 0002:0004       rsrvptrs
 0001:0032       STGCREATEDOCFILE
 0001:0058       STGCREATEDOCFILEONILOCKBYTES
 0001:00DA       STGISSTORAGEFILE
 0001:0100       STGISSTORAGEILOCKBYTES
 0001:007E       STGOPENSTORAGE
 0001:00AC       STGOPENSTORAGEONILOCKBYTES
 0001:0126       STGSETTIMES
 0002:0010       STKHQQ
 0001:0006       WEP
 0002:00C0       _edata
 0002:00C0       _end
 0000:9876  Abs  __acrtmsg
 0000:9876  Abs  __acrtused
 0000:9876  Abs  __acrtused2
 0000:D6D6  Abs  __aDBdoswp
 0002:0012       __adbgmsg
 0002:001A       __aDBrterr
 0002:002A       __caption
 0002:00C0       __edata
 0002:00C0       __end
 0000:9876  Abs  __fptaskdata
 0001:0164       __NMSG_TEXT
 0001:019B       __NMSG_WRITE
 0001:0161       __wflags
 0000:0000  Imp  __WINFLAGS           (KERNEL.178)
 0002:001C       ___aDBexit
 0002:0018       ___aDBswpchk
 0002:0016       ___aDBswpflg

  Address         Publics by Value

 0000:0000  Imp  CALLPROC32W          (KERNEL.CALLPROC32W)
 0000:0000  Imp  LOADLIBRARYEX32W     (KERNEL.LOADLIBRARYEX32W)
 0000:0000  Imp  OUTPUTDEBUGSTRING    (KERNEL.115)
 0000:0000  Imp  GETVDMPOINTER32W     (KERNEL.GETVDMPOINTER32W)
 0000:0000  Imp  __WINFLAGS           (KERNEL.178)
 0000:0000  Imp  FREELIBRARY32W       (KERNEL.FREELIBRARY32W)
 0000:0000  Imp  GETPROCADDRESS32W    (KERNEL.GETPROCADDRESS32W)
 0000:0000  Imp  CALLOBJECTINWOWCHECKTHKMGR (COMPOBJ.204)
 0000:0006  Abs  pLocalHeap
 0000:0008  Abs  pAtomTable
 0000:000A  Abs  pStackTop
 0000:000C  Abs  pStackMin
 0000:000E  Abs  pStackBot
 0000:9876  Abs  __acrtmsg
 0000:9876  Abs  __acrtused2
 0000:9876  Abs  __fptaskdata
 0000:9876  Abs  __acrtused
 0000:D6D6  Abs  __aDBdoswp
 0001:0000       LIBMAIN
 0001:0006       WEP
 0001:000C       DLLGETCLASSOBJECT
 0001:0032       STGCREATEDOCFILE
 0001:0058       STGCREATEDOCFILEONILOCKBYTES
 0001:007E       STGOPENSTORAGE
 0001:00AC       STGOPENSTORAGEONILOCKBYTES
 0001:00DA       STGISSTORAGEFILE
 0001:0100       STGISSTORAGEILOCKBYTES
 0001:0126       STGSETTIMES
 0001:0161       __wflags
 0001:0164       __NMSG_TEXT
 0001:019B       __NMSG_WRITE
 0002:0004       rsrvptrs
 0002:0010       STKHQQ
 0002:0012       __adbgmsg
 0002:0016       ___aDBswpflg
 0002:0018       ___aDBswpchk
 0002:001A       __aDBrterr
 0002:001C       ___aDBexit
 0002:002A       __caption
 0002:00C0       __end
 0002:00C0       _end
 0002:00C0       __edata
 0002:00C0       _edata
